:030000000219FDE5
:03000B000200AA46
:03002B0002015679
:03005B000202DFBF
:030073000202CCBA
:1000800002030406080C10182030406080040608A3
:100090000C10182030406080A0C00003070F1F0D17
:1000A0000D04050D050205030302C2AFC0D0C0E078
:1000B000206214E5256009E473E525F4F58AD2622F
:1000C000D0E0D0D0D2AF3285268AC262E526F46075
:1000D00029D0E0D0D0D297D295D293D2AF32D29756
:1000E000D295D293206F0C2065097405D5E0FDE50B
:1000F0007B4290D0E0D0D0D2AF32758A00C28DD290
:100100006201F301B9306805206502C29701B93078
:100110006805206502C29301B9306805206502C2F6
:100120009501B9C29630680A206507740FD5E0FDC5
:10013000C29701B9C29230680A206507740FD5E0F2
:10014000FDC29301B9C29430680A206507740FD5C7
:10015000E0FDC29501B9C2AFC2AD53E6EFC0D0C059
:10016000E0D2D3D2AFC2CEE52A6007207449152A67
:1001700021B77800790020742EE580307E01F430BC
:10018000E50278FF53DACF207E0343DA20307E0386
:1001900043DA10C2D8C271E580307E01F430E50246
:1001A00079FFC3E89970CB306103752A1820740376
:1001B000752A18885CD27020740DE52B6004152B0D
:1001C00021C743DA01C2D82070024136A85C206101
:1001D00002C2702074367982B70431C3E894F040CB
:1001E0000374F0F8E8C4540F28F87984B703024187
:1001F0000CC313C3138721200802C313200A06C3AC
:10020000C898F8410C28F8500374FFF88822E52DAF
:1002100054066022206B1FE536C333C333F8E56410
:10022000C313C313F9C3952240028922E82522F59E
:100230002250037522FF7882B6044E852224A8241A
:10024000C3E52495614002A861C3E895634002A814
:10025000638825E56670024187C3E8AA669A500361
:10026000E8FAE4F9EAC333FBE568F45B29400D25BD
:1002700067F8E56760021567400B41870AC3E567C9
:100280009A5002056778FF882620CF0AD0E0D0D0A8
:1002900043E610D2AD32C2CF053A7801E52A6005B7
:1002A000307402152AC3E55C94014005755F004176
:1002B000C2756000756900E55F2401F55F50037544
:1002C0005FFFD0E0D0D043E610D2AD32C2AF53E6EC
:1002D0007F7592FA7593FFC260759104D2AF32C2F6
:1002E000AF53E6EFC2ADC0D0C0E0C0F0D2D3D2AFC2
:1002F000A8FBA9FCC2D8307102614653DACF207E38
:100300000343DA10307E0343DA20D271E580307E79
:1003100001F420E502611D88278928A17353DACFF3
:10032000207E0343DA20307E0343DA10C2D8C27144
:10033000307402A15F7800E580307E01F430E50280
:10034000A15F885CA14753DACF207E0343DA2030D7
:100350007E0343DA10C271206102811F53DACF207D
:100360007E0343DA10307E0343DA20C2D8D271888C
:10037000578958C3E89555F8E99556F97B007E08EA
:100380007A00C3E8948CE994005005755B008111F4
:10039000882178A2E6A8216055C3E894C8E99400B2
:1003A0005008E4D2E4FB7A0A61ECC3E89468E9946B
:1003B000015008E4D2E3FB7A0F61ECC3E894D0E982
:1003C00094025008E4D2E2FB7A1E61ECC3E894A0E8
:1003D000E994055008E4D2E1FB7A3C61ECC3E8946F
:1003E00098E994085008E4D2E0FB7A787E00C3E8EC
:1003F0009559FCE9955AFD30E70AECF42401FCED2F
:10040000F43400FD755B00C3EC9AED9E5003755B00
:10041000018859895A8557558558567802A147C38E
:10042000E89527F8E99528F9307C02A12B307B026A
:10043000A12B307A02A1242075028142E9FDE8FC5B
:100440008161E9C313F9E813F8307902A124E9C303
:1004500013F9E813F8307802A124E9C313FDE81377
:10046000FC20612CC3EC941CED940240028178EDD9
:0E047000701EC3EC94C850180529E5297002CF
:10047E001529C3E529940A5002A15F755C00D2705C
:10048E00A15FE529600215297888E6F97400207FBE
:10049E00087896B90302789EE624FAFEE43400FF4B
:1004AE00C3EC9EFCED9FFD9208B90310A208500705
:1004BE00207609D27681CA307602C276A20850160C
:1004CE00B9030DECF42401FCEDF43400FD0204E458
:1004DE0078007900A12BB90315EC33FCED33FDC385
:1004EE00EC940AFCED9400FD50047C007D00C3ECFE
:1004FE0094FFED9400400678FF7900A12BEC8572F5
:10050E00F0A4C5F0A2F733F879004003020547784E
:10051E00FF7900020547E9C313F9E813F8307C0EA2
:10052E00E9600278FFC3E81338F8E43400F9C3E851
:10053E0094FFE99400400278FF885CD2702061023B
:10054E00A15F741FF4552F4BF52FC274EB7002D2BE
:10055E0074752A18307403752A0A306102A173204B
:10056E00740353DAFE207403752B06D0F0D0E0D05E
:10057E00D0D2AD43E6103279010205A3790302050C
:10058E00A3790A0205A3791E0205A379640205A3C5
:10059E0079C80205A37817E4D5E0FDD8FAD9F6227A
:1005AE007A147B780205CA7A107B8C0205CA7A0D02
:1005BE007BB40205CA7A0B7BC80205CAE573D5E087
:1005CE0001227902E4C292D5E0FDC293D5E0FDD2BC
:1005DE0093D5E0FDD292D5E0FDE920E002C297303E
:1005EE00E002C295E573D5E0FDE920E002D2973036
:1005FE00E002D2957496D5E0FDD9C9EAF8D5E0FDB2
:10060E00D8FBDBB8C29222C37C007D0075F00005DA
:10061E00F0EA33FAEB33FB50F6EB13FBEA13FAC3B3
:10062E00E9FFE8FEE89AF8E99BF95004EFF9EEF8D5
:10063E00B3EC33FCED33FDD5F0DFEDF9ECF822E849
:10064E0089F08A20D2D4F8A9F07B0030F70B7BFF1B
:10065E00F42401F8E9F43400F9E88520F0A4ADF0B3
:10066E00F8E98520F0A4AFF0FEED2EF974003FFA04
:10067E007C04C3EA13FAE913F9E813F8DCF48BF0FF
:10068E0030F70AE8F42401F8E9F43400F9E889F0C7
:10069E00C2D4F8A9F0227882B604030206FFC3E59D
:1006AE005C940140030206C9852224E4F544F54515
:1006BE00F546F547F548C26E0206FF7882E6FCD293
:1006CE006EE522F523783879C7AA40AB41C3EB1308
:1006DE00FBEA13FAEC146013C3EB13FBEA13FAEC08
:1006EE0014146007C3EB13FBEA13FAD1158844897F
:1006FE004522C3E5449523F8E5459400F9500CC313
:10070E00E89480E994FF4016020730C3E8947FE92D
:10071E0094005003020730787F790002073078800A
:10072E0079FF8849894A22E5492546F8E54A354741
:10073E00F9854A20E4300701F43548FA30E709C359
:10074E00EA94F0401502076EC3EA940F50030207B5
:10075E006E78FF79FF7A0F02076E780079007AF0D3
:10076E00C3E5249561500AC374019524500B02070A
:10077E008CE54A20E70E02078CE54A30E7068846EC
:10078E0089478A482278A5E6FAC3E54933F8E54A4F
:10079E0033F9D14DE930E70BC3E89480E994FF407B
:1007AE0013E1C6C3E8947FE994005002E1C6787F56
:1007BE007900E1C6788079FFE820E715C3E5239834
:1007CE00F84009C3E8940140030207ED78010207DF
:1007DE00EDE8F424012523F840030207ED78FF88A5
:1007EE004B2278A6E6FAA847A948D14DE930E70C86
:1007FE00C3E89401E994FF4016020821C3E894FF70
:10080E00E99400500302082178FF7900020821784C
:10081E000179FFE920E715C3E54B98F84009C3E8D5
:10082E00940140030208487801020848E8F42401C4
:10083E00254BF8400302084878FF88242278FF20D1
:10084E00692879A1E76023E541601F74FF8541F0B7
:10085E00848539F0306A0375F005A4F8C5F060029E
:0E086E0078FFC3E895645002A864886322C333
:10087C00E5409440E5419401E563500314018C0478
:10088C006002F563220208942275E890227883E6D0
:10089C00FF30EDF9A8BDA9BE0570C3E57094084002
:1008AC0052757000E9FA79A0E76044EA7007E571C7
:1008BC00601B0208CDC3E895716010E571500660AD
:1008CC000C140208D90460F90208D9E571F571C35A
:1008DC00946D401B7561C0C394044013756180C353
:1008EC009404400B756140C394044003756100751A
:1008FC00BB0822E5612410500274FFF5617982B7C0
:10090C0004022126C3A861E524985002A824C3E858
:10091C0095634002A86388258826E570B4070375A3
:10092C00BB1022743279A787F0A4C5F0A2F733F874
:10093C00C3E895614002A86188228824882588260E
:10094C008864227540007541F022C2AF75C820A89A
:10095C00CCA9CDAA3A30CF010A75C824D2AFAB3B93
:10096C00AC3C883B893CC3E89BF8E99C206908F9BE
:10097C00306602416521BFAD3D8A3DF9EA9DFA60C2
:10098C000478FF79FFAE3EAF3F8B3E8C3FA83BA96E
:10099C003CC3E89EF8E99FF9C3E54113FBE540131E
:1009AC00FAE82AF540E93BF54150067540FF7541E0
:1009BC00FF410CAA40AB41AC40AD417E047F02C369
:1009CC00EB9404400D1E1FC3EB94084005206A02F3
:1009DC001E1FC3ED13FDEC13FCDEF7C3EA9CFAEB10
:1009EC009DFBEF6009C3E913F9E813F8DFF7EA2878
:1009FC00FAEB39FB8A408B4150067BFF8B408B41D5
:100A0C00C3EB94025002D2663069047F03413778FD
:100A1C0092E6FFC3E537948240110FC3E53794A0EB
:100A2C0040010FC3EF940640027F057E02E541C4EE
:100A3C00540FF9E541C454F0F8E540C4540F28F8BC
:100A4C00C3E89EFAE99400FB4009C3EA9402EB94D4
:100A5C000050047A02E4FB41B1AA40AB41EBC4FE66
:100A6C00EAC4540F4EFCC3EA9CFAEB9400FBC3E8B7
:100A7C0013C313F8EA28FAEB3400FB8A408B41C30A
:100A8C00EB94024002C2667802EBC4FE7B00EAC41F
:100A9C00540F4EFAC3EA98FA4005C3940250027AF6
:100AAC00027892E6FF30600241B1855192855293F3
:100ABC00D26043E680C3E49AF8E49BF930660261A5
:100ACC003DE8FAE9FBD3E913FDE813FC88518952A0
:100ADC00C3EF94036038EF20E00DE82CF8E93DF902
:100AEC00ECFAEDFB020B06E828F8E939F9C3E82427
:100AFC0002F8E93400F97AFE7BFFC3EF9403400E51
:100B0C008A538B54884D894E8C4F8D50617188530C
:100B1C0089548A4D8B4E8C4F8D503069127553F021
:100B2C007554FF754FF07550FF7551F07552FF619C
:100B3C0071E8FAD3E813FC8851C3EF94036020EFFB
:100B4C0020E007E82CF8ECFA615DE8282402F87A3A
:100B5C00FEC3EF940340088A53884D8C4F61718813
:100B6C00538A4D8C4FE568C3335002646BF5683083
:100B7C006002617B753402D26043E680E52D540639
:100B8C006034A840A941C3E913F9E813F8C3E91389
:100B9C00F9E813F8306904E92440F9C2AF53E67F51
:100BAC00759100C3E498F594E499F595759104D288
:100BBC006043E680D2AF22D26475430075200030CA
:100BCC006C03752040020BE2D26475430075204023
:100BDC00306C0375200078017901206620E52D54D6
:100BEC00066002C2647914E541C313700104F8C3B2
:100BFC00941440027814306904781B791B2060101F
:100C0C00E543600C306903D53404D26D818C71835B
:100C1C000543E59B5440B52002817630690908C331
:100C2C00E899400118810920640A08C3E899400238
:100C3C0061E28109C264C2AF53E67F7591003066F0
:100C4C00127594007595F8759104D26043E680D2C4
:100C5C00AF61E2E5417EFFC3334005C3334001FE83
:0F0C6C00C3E49E759400F5958153C3E53394015D
:100C7B00500261E230640261E2D802818A8109C2CA
:100C8B006DC2AF53E67F759100855394855495756E
:100C9B009104854D92854E93D26043E680D2AFE5A9
:100CAB002D54066008206A020533020CC8306D0D06
:100CBB00206C0A20640715811581021572227800B9
:100CCB003064027801E53775F007A4F9E5F028F5F3
:100CDB00F0E9A2F013A2F113A2F213F537C3947843
:100CEB005003753778C3E53795384008D265D297EE
:100CFB00D295D29330600281FF854F92855093D26B
:100D0B006043E68022207D16C2AF754202C292D2AA
:100D1B0096306202C295D2AF759F13020EFFC2AF1F
:100D2B00754202C292D294306202C297D2AF759FC3
:100D3B0013020EFF307243207D20C2AF7542039029
:100D4B000134757B04D295C294306204C293A15DC9
:100D5B00D292D2AF759F10020EFFC2AF75420390B5
:100D6B000134757B04D297C296306204C293A17D85
:100D7B00D292D2AF759F11020EFF207D17C2AF75B5
:100D8B00420390010FD295306202C293D2AF759F8E
:100D9B0010020EFFC2AF75420390010FD297306263
:100DAB0002C293D2AF759F11020EFF207D16C2AF08
:100DBB00754204C296D294306202C293D2AF759F31
:100DCB0011020EFFC2AF754204C294D2963062027A
:100DDB00C293D2AF759F10020EFF307243207D205D
:100DEB00C2AF754205900123757B40D293C29230FE
:100DFB006204C297C103D296D2AF759F13020EFF46
:100E0B00C2AF754205900145757B10D293C29230EB
:100E1B006204C295C123D294D2AF759F13020EFF09
:100E2B00207D17C2AF754205900105D29330620247
:100E3B00C297D2AF759F13020EFFC2AF75420590DA
:100E4B000119D2933062EBC295D2AF759F13020E8C
:100E5B00FF207D16C2AF754206C294D29230620259
:100E6B00C297D2AF759F10020EFFC2AF754206C27A
:100E7B0096D292306202C295D2AF759F11020EFFCD
:100E8B00307243207D20C2AF754201900145757BC6
:100E9B0010D297C296306204C295C1A9D294D2AF38
:100EAB00759F11020EFFC2AF754201900123757B36
:100EBB0040D295C294306204C297C1C9D296D2AFC8
:100ECB00759F10020EFF207D17C2AF754201900176
:100EDB0019D297306202C295D2AF759F11020EFFE5
:100EEB00C2AF754201900105D295306202C297D212
:100EFB00AF759F10C26522900103757B00D297D20C
:100F0B0095D293C296C294C292C26222788076091D
:100F1B000876090876040876FF0876030876FF083A
:100F2B00760B087601087601087601788C76010835
:100F3B0076FF0876FF0876FF0876FF0876FF0876BF
:100F4B00030876FF0876FF0876FF0876250876D02B
:100F5B000876280876500876040876FF087602088B
:100F6B00760008767A0876FF08760108760108760F
:100F7B0000087603087600227887E6FFC27278882D
:100F8B00E6C394036008C27DE630E102D27DC27EE7
:100F9B007889E630E102D27EC3EF94026008758E49
:100FAB0001D273020FB6758E00C273227880E614DD
:100FBB009000809378A5F67881E614900080937862
:100FCB00A6F67886E61490008D9378A7F67886E6D9
:100FDB00F539C394025003753902789CE67538FFD6
:100FEB00B402037538A0B4030375388278A3E614F2
:100FFB0090009A93F566120F0222227896E6FA7801
:10100B0097E6FB7888E6B40305C3EB940EFB307FC1
:10101B00047A007BFFC3EB9AFCC3948250027C8260
:10102B007572000572EC8572F0A4C3E5F0947D40F7
:10103B00F222D27F11061205941205947A007B00DE
:10104B007C1012058AE55C2AFA74003BFBDCF37C0E
:10105B0004C3EB13FBEA13FADCF7FEC27F11062283
:0E106B00757C00757D00E5EF20E60375200022
:101079000520903FFFE520146006901DFF146000D5
:101089009304600375EF1653D9BF7581C043FF8080
:1010990012058575EF0643B203E5B3240220E70D77
:1010A900F521E5E320E0068521B343E301120F02B0
:1010B9007580FF75A40075F1B275D4DF7590A975B7
:1010C900A5FC75F2FE75D50175A60175E241120FF1
:1010D90002E4F8F6D8FD756801120F171215C378E6
:1010E900988673753001C2AF12059E1205AE1205BE
:1010F900941205B51205941205BC120594C2AF7578
:101109007C00757D0078FA79FA308507D9FBD8F724
:10111900021C00120F83120FB71105110678988669
:1011290073120F0275881075890275C824759104A8
:1011390075D84075A82275B80275E690759B8075BB
:101149009D0075D10E75BC5875BB0875BA1175E847
:1011590080120585D2AF12089175360053DACF2077
:101169007E0343DA20307E0343DA1043DA01C2D822
:10117900C27112059ED2617B037A0CE55B70077A16
:101189000CDB03021106120594207003021106C23A
:1011990070E55CC3940240E1E52F541F855E5DF55F
:1011A9005EB55DD5DAD5C26153DACF207E0343DA65
:1011B90020307E0343DA10C2D8C27178A2E67008E3
:1011C900D274E52F54E0F52FC275752900120599DF
:1011D900307409C3E529940A4002D27512058A7848
:1011E900023074027800C3E55C9840F0C2AF120582
:1011F900AE1205AE1205AED2AF12059E754C00783F
:1012090088E6B4030241FB12058A788CE6C394018F
:1012190050030212FBE530C3940150030212FB751F
:101229007CA5757DF1207435C3E55C94FF500302FC
:1012390012FBC2AF1205C3D2AF120599C3E55C9484
:101249000150EFC2AF1205AE12058F1205AED2AF33
:10125900120599C3E55C94FF40E902176F7F02D23A
:101269007F1106120599C2AFC27F1106AE5CC3E5B4
:101279005C947FD2AF5002610B120585C2AF120593
:10128900C3D2AFDFDA113DC3EE7897F612059E128D
:1012990016F27F0AD27F1106120599C2AFC27F11D9
:1012A90006AE5CC3E55C947FD2AF50E6120585C2F9
:1012B900AF1205AE12058F1205AED2AFDFD6113DC2
:1012C900EE24037896F6F87997E7C3948240039859
:1012D9005006E824827897F612059E121605121711
:1012E900211205991106C3E55C94FF5002412802B9
:1012F900176F757C00757D00C3E55C954C400385CF
:101309005C4C12059978017988E7B403027805C322
:10131900E55C9840024108C2AF1205C31205C31229
:1013290005C3D2AF12059E753000E4F531F53205DB
:1013390031E531F4703F0532789AE6781914601274
:10134900783214600D787D14600878FA146003759A
:101359003200C3E53298401D120F0212058515327D
:1013690075310078998673C2AF1205C3D2AF7898E8
:10137900867312059912058FE52A700530740221CA
:101389000678012074027806C3E55C9840A1788844
:10139900E6C394036003120599E52A700302110656
:1013A900C2AF120F02E4F522F523F524F525F5263F
:1013B900F567D2AF7885E6C333F565E4F544F545BD
:1013C900F546F547F548F570F52CF52DF5377570A7
:1013D9000875BB1012058512089530EDFDA8BDA949
:1013E900BEE97001F8887112089975700875BB100B
:1013F900120F83C2AF7561FF12092F852261852201
:1014090062852263D2AF75220175240175250175A4
:101419002601856069756A017888E6B40307C27D8B
:10142900307602D27DD268D269753300120E5C1211
:101439000E8B12094F12095612094F120956120939
:101449004F120BD41206A4120CC9120D1012095610
:10145900120BC3306E0312070020660312084B30CB
:0E146900660312087B120CC9120D3F120956C1
:10147700120BD4306E03120735120CC9120DB612B7
:101487000956120BC3306E03120793120CC9120DC3
:10149700E5120956120BD4306E031207F0120CC96D
:1014A700120E5C120956120895120BC3120CC912C0
:1014B7000E8B12089912095630693285646185646A
:1014C70062856069756A0179187A0CC3E5339940BA
:1014D7000FC269D26A8A358564618564630214F430
:1014E700C3E55C9401400302144A02157A306A1D71
:1014F700206C1AE535147006C26AD26B814AF5353D
:10150700C3E55C9401400302144A02157A7536005C
:1015170078FA79A4E760027803C3E55F98505430FE
:101527007404E52A604D7888E6B40317207D05200A
:101537007607A14A307602A14A206C07D26C8564EF
:1015470061818978F0306C058564617820C3E54155
:10155700985002814A306C1BC26CC27D307602D231
:101567007DD26A753512856461814A0536E55C600E
:1015770002A17D753600C2AF120F027887E6FE76AC
:1015870002120F837887EEF6E4F522F523F524F5AA
:1015970025F526F565752C00752D00D2AF12059936
:1015A700120F0278A4E66006C297C293C295307400
:1015B70009C3E5369404400221066133901A0D7879
:1015C70020121647E520B4550CA3121647E520B4A0
:1015D700AA030215E5120F17121605021604901A30
:1015E7000378807B0A121647A308DBF9901A0F7855
:1015F7008C7B19121647A308DBF9901A2822C2AF71
:1016070012168A121667901A00740E12164CA374DB
:101617000712164CA3741512164C901A0378807B88
:101627000A12164BA308DBF9901A0F788C7B191254
:10163700164BA308DBF912169D12167B901A282267
:10164700E493F622E6438F01538FFDFFC3E58394AE
:101657001C400122EF857CB7857DB7F0538FFE22B2
:10166700438F02438F01857CB7857DB7901A0DF0B4
:10167700538FFC22901A0D7455D14C901A0E74AAF0
:10168700D14C227A3079D07820901A40D147E52082
:10169700F709A3DAF7227A3079D0901A40E7D14CCC
:1016A70009A3DAF922AB74A875BB01027980BB02E2
:1016B700027981BB03027982BB04027984BB0502EC
:1016C7007986BB06027992BB07027987BB08027944
:1016D700A3BB0902799CBB0A027988BB0B027989F3
:1016E700E8F7227C0512059EDCFB22C2AF1205AE8D
:1016F7001205B51205BC1205C312058F1205AE12ED
:1017070005B51205BC1205C312058F1205AE1205E9
:10171700B51205BC1205C3D2AF22C2AF1205C31260
:1017270005BC1205B51205AE12058F1205C31205C9
:10173700BC1205B51205AE12058F1205C31205BC02
:101747001205B51205AED2AF22AE74AF75C2AF1295
:1017570005AE1205AE1205AE12058FDEF21205C3F5
:1017670012058FDFF8D2AF22D1F2D1EAD1EA757430
:1017770001757501757600F1507C05AD5C12059E0B
:10178700C3ED955C70F5C3E55C9401400AC3E55C65
:1017970094FF40320217ABD1ACD105D1F2C2AF757D
:1017A700EF16D1EADCD50576C3E5769403500280BF
:1017B700C6D1EA0575E5741490009F93F808C3E550
:1017C7007598500280AED1EAD1EA0574C3E57494E6
:1017D7000C5002809C120F17D105C2AF75EF16D1BE
:0117E700EA17
:0319FD0002106B6A
:101A00000E0715090904FF03FF0B01010155AA0187
:101A1000FFFFFFFFFF03FFFFFF25D0285004FF0259
:091A2000007AFF0101000300FF40
:101A4000235475726E696779364123202020202047
:101A500023424C48454C4923463333302320202031
:101A60002020202020202020202020202020202076
:101C0000C2AFC2D353D9BF7581C043B20343FF8073
:101C1000752438752503B1DC7529A5752AF175E29F
:101C20004043F12053A4DF75D4FFD2857DFA7803B9
:101C300079E67C10752200752300901DE97B0675FE
:101C400024987525013085028145208508D8FBD967
:101C5000F9DCF781B7308508D8FBD9F9DCF781B713
:101C6000B19CE493A3C39A6004DDC381B7DBDBB10D
:101C70008E6002812E7B08E493FAA3B16FDBF87AC1
:101C800030B16F752200752300B18EEAFCEBFDC305
:101C9000ED94FE400EB18E8A278B28ED30E0048A49
:101CA000828B83B18E7AC270D8C3ED94FE601950D6
:101CB000CEBD002BEC600F7520007521FF7529004B
:101CC000752A000200008100A827A9280809D80465
:101CD000D90281DCB192EA89AAF281CE0D81A3C337
:101CE000ED94035053EDA2E092007AC5C3E58294CF
:101CF00000E583941C508A200010438F02438F011B
:101D00008529B7852AB7F0300029A827A92808090E
:101D1000438F01538FFDD804D902A133C3E58394C7
:101D20001C4003A3A11689AAE28529B7852AB7F02A
:101D3000A3A116538FFC817F7AC1BD030CE493A34A
:101D4000FAB153DCF8B14B817F8181AA22AB23B178
:101D50006FEBFAEA6222752608C3E52313F523E543
:101D60002213F52250066323A0632201D526EAB18F
:101D7000DCB1DC75260AEAF4200102D285300102CA
:101D8000C285B1DCC3134002C201D526EB22B19259
:101D9000EAFB208502A192308502A197752608AE44
:101DA00024AF25C3EF13FFEE13FEB1E0B1DCC3EAAD
:101DB000133085024480FA30E703632201C3E52330
:101DC00013F523E52213F52250066323A0632201B5
:101DD000D526D9E52265236523F52222AE24AF2539
:101DE0000E0FDEFEDFFCD20122424C48656C6934E6
:071DF000373163F3300601F7
:00000001FF
